:1000000028C9189518951895189518951895189544
:100010001895189518951895189518951895189578
:10002000189518951895D4016000821D6600340259
:10003000000003E312D003E31CD000E012E3A9D0D8
:1000400003E30FD002E00DD008E00BD001E005D0B3
:1000500006E007D00CE00DD008950BD006D005D0F7
:10006000089507D000E812E094C000E01DE791D0A9
:1000700008958A93802F949800E410E010D0082F00
:1000800002950F7012B3102B12BB0ED008D08F70D8
:1000900002B3082B02BB08D07CD08991089579D097
:1000A00002B3007F02BB0895959A00E410E071D07E
:1000B000959800E411E008958A93802F949ADCCFFC
:1000C00011D0D80180E003C012D0F6DF839590E014
:1000D0000ED0002311F08131B8F389919991A99143
:1000E000B9910895BA93AA939A938A930895FD01BA
:1000F000E80FF91F00810895F5DF00E4BADFAFEFE4
:1001000090E002C0A6959395983098F4BA2F80E0BD
:1001100004C000E0D1DFB6958395883098F7BB2303
:1001200011F001E001C000E010E0012B91F70FE1B8
:10013000F1CFD3CF8A9304E105BD80E001C006D0A2
:100140008630E8F300E005BD8991089500E61AEED7
:1001500020D0839508958A9303E105BD80E001C016
:10016000F5DF8730E8F304E105BD80E001C0EEDF94
:100170008730E8F305E105BD80E001C0E7DF8730A7
:10018000E8F303E105BD80E001C0E0DF8730E8F37C
:10019000D9CF01501040202F212BD9F7089510E01E
:1001A0001FBB0EBBE09A0DB30895202F30E03FBB7C
:1001B0002EBB1DBBE29AE19AE199FECF08950BD0C8
:1001C000089500E0022B132B0F531240212F220F12
:1001D000220B322F089504B1202F30E015B100E03A
:1001E000022B132B0895BA93AA933CD03ED041D052
:1001F0006ED0012B89F000814AD0A801B901DB0142
:100200004AD065D044D07B2FCDD740E050E060E7A6
:1002100072E4F8D934D945D046D051F423D0E8E778
:10022000F2E046D059D042E03AD059D05BD045D028
:1002300019D0E8E7F2E046D055D00DD02E3500E0D9
:10024000300714F003E603D0A991B991089510E0A6
:1002500039C000831183202F312F0895EEE7F2E09B
:1002600036D0C8013FD033D00895EAE7F2E02AC083
:1002700033D0ECE5F2E0089538D029D03AD0F3D865
:10028000CFDA40E050E060E070E4BCD9089531D0AE
:10029000EAD8089521D0E0E5F2E008954EE02AD0B2
:1002A000089520D00FC000919502013008951DD00F
:1002B000208131810895201B310B208331830895E3
:1002C000E5E8F2E0008311830895E0E8F2E00081C0
:1002D0001181089520813181021B130B0895200F95
:1002E000311F0895E4E7F2E00895ECE7F2E00895A5
:1002F00012406CCF50E019C87A926A925A924A9290
:10030000AA939A938A930FE301BBB99ABA9ABB9ABC
:100310008E9A8F9AA99AAA9AAB9AAC9A379A369AD9
:10032000359A33983298319A309A00E007B9479A53
:1003300080DEE2DE03E212E0CBD620E630E0CFD66C
:10034000CAD6BEDE23E630E05BD601C02CD68035AF
:1003500000E09007D8F3969A979A2BD6FCDE29D620
:100360009698979800E11BDF0F3FD1F413E000E16E
:100370001CDF10EE01E119DF11E002E116DF12E0EF
:1003800003E113DF10E0B7D610E0B8D612E0B9D61B
:1003900010E0BAD610E00AE108DF12E80BE105DF51
:1003A00000E1FDDE902F80E001E1F9DE10E0082B96
:1003B000192BD5D687DF02E1F2DE00938D0203E12F
:1003C000EEDE00938E0204E1EADE00938F0205E187
:1003D000E6DE0093900206E1E2DE0093910207E17F
:1003E000DEDE0093840208E1DADE10E069DF09E175
:1003F000D6DE009394020AE1D2DE802F90E00BE17A
:10040000CEDE302F20E0282B392B80D656DFC19A44
:10041000C29800E50FBD09E00EBD00E010E01DBD73
:100420000CBD3CD61695079519BD08BDCBD500E08F
:100430000093880200938902CAD500E000938C02E1
:1004400000939602009395020093920200938B0210
:10045000009393020CEE1FEF33DF08EDEAE6F2E0C3
:1004600031DF04E110E0ECE6F2E02CDF03E6FDDE34
:1004700018DFD6D568D64BE050E03ED7E2E8F2E090
:1004800021DF00912802003509F052CF80E006C03C
:1004900096DE0F531240FFDE15DF0196883E03E023
:1004A0009007B0F3B5D50CC004B110E035B120E031
:1004B000202B312BDEDE0BDF020F131F03DF019633
:1004C0008A3000E0900780F3D4DE0081102F0DE128
:1004D0006CDE009127020B3409F02ACF00E010E017
:1004E00020E030E044D6EEDE2283338343D6EADEDA
:1004F0002283338300919302005049F00A9561F101
:100500000A9509F44EC00A9509F470C097C080D5C9
:1005100007C02CD532D5B19902C0B299FACF019655
:10052000C1D508F08BC03698369A01C017D5B19B5B
:1005300002C0B299FBCF3698369A02C00FD511D5BA
:10054000B19B02C0B29BFACF3698369AB199E3CFED
:10055000B299E1CF06D5FACF5BD507C007D50DD547
:10056000B19B02C0B299FACF01969CD508F066C043
:100570003698369A01C0F2D4B19B02C0B29BFBCF31
:100580003698369A02C0EAD4ECD4B19902C0B29B34
:10059000FACF3698369AB199E3CFB29BE1CFE1D446
:1005A000FACF36D507C0E2D4E8D4B19B02C0B29BE3
:1005B000FACF019677D508F041C03698369A01C037
:1005C000CDD4B19902C0B29BFBCF3698369A02C007
:1005D000C5D4C7D4B19902C0B299FACF3698369A29
:1005E000B19BE3CFB29BE1CFBCD4FACF11D50BC006
:1005F000D6D4C0D58ED5D3D4BAD58BD5B19902C0B7
:10060000B29BF6CF01964ED5C8F43698369A01C003
:10061000B7D4B19902C0B299FBCF3698369A02C0CE
:10062000AFD4BAD4B19B02C0B299FACF3698369AF9
:10063000B19BE4CFB299E2CFAFD4FACF9BD51BD513
:1006400011950195104068D53DDE91D514D56BD537
:1006500039DE62D53CDEECE4F2E034DE60D5E8E57C
:10066000F2E030DE00918702002361F000E00093A9
:10067000870252D52CDEEEE6F2E024DE50D5E0E72C
:10068000F2E020DEEEE6F2E022DE46D511DE13DEF9
:10069000E0E7F2E01CDE47D50BDE0DDE58D569F44D
:1006A000E1D4E2E5F2E01BDE08DE36D510DEF2DD55
:1006B000C8D435D5DDDD06DE11C0013079F4D2D4E1
:1006C0000EDEE9DDFADD022F132FE2E5F2E0B9D408
:1006D000822F932F0197CDDD80839183CADD8081A6
:1006E0009181D9DD78D4E5E8F2E050D51ED6801BA3
:1006F000910BE4E6F2E08083918300E010E0F5DD09
:10070000E1DD14D509F0EBC000918802013009F059
:10071000E6C0022F132FC2DDE6E6F2E0D3DDA9DD4D
:10072000D6DDBCDDE8E6F2E0CDDDE6E6F2E0CFDDE9
:1007300092DD309F302D219F300D209F202D310DD7
:10074000E8E6F2E023D5042F152F149F102D059F06
:10075000100D049F002D110D020F131F98DD9CD961
:100760008ED6C3DDAFDD312F332312F402ED03C08B
:10077000012B11F401E06BDD9BDD293C00E030072B
:1007800034F00FE105BD00EB03BD13D4ACC0009104
:100790008D0210E06EDD8CDD021713070CF08BC0AC
:1007A000E4E6F2E085DD021713070CF084C0A0E058
:1007B0009CDD7ED487DDCBD451F4AED47DD478DDFE
:1007C00069DD80DDB0D47CD473DD52DD7BDD0BDDF3
:1007D00000918D0210E05FDD6BDD02171307E4F579
:1007E0000023D1F13BDD4AE05ADD402FA3D4A1F52F
:1007F00039DD3BDD58DD39F40ED40E5F03BD02E375
:1008000010E0C7DC6CC000918F02002319F403D400
:100810000D5FF4CF013089F40CE105BD63DD00818B
:10082000000F065F03BD00E315E7B3DC5BDD00816D
:10083000065F03BD00E117E2E4CF023009F04FC0CC
:100840000DE605BD84E190E0863E00E0900708F0EB
:1008500046C0D1D3AAD3F8CF00918E0210E01195F3
:100860000195104020173107D4F5F8DC4CEE5FEF0E
:100870005CD5402F455F5ED491F500918E02002338
:1008800071F1F0DCF2DC00918F02023069F40BDDD3
:1008900059F00EE605BD84E190E0863E00E0900749
:1008A000F0F4A9D382D3F9CF0EE6B6D3039503BDF6
:1008B00004EF11E0A6CF00E005BDC398E4E5F2E047
:1008C000FBD300DD29D403DDE4E5F2E0FBDCE0E668
:1008D000F2E0F6D3F7DC23D4E0E6F2E0F3DCEAE77B
:1008E000F2E0F5DCDEDC99992CC06DD300938A022E
:1008F0008FD30CE0BEDB999917C055D38E3200E040
:100900009007C8F300919602009500939602002389
:1009100011F400E001C006E0009395020BDC00E753
:1009200017E137DC45D367C101D421F480D302300D
:1009300038F003C07CD3073018F000E00093950234
:1009400050C19A9979C0A0E0F1D361F000D451F47C
:10095000E3E9F2E06ED3043018F000E00093930274
:10096000E9DB49C1F8D3F1F4D1D3B1DC40918B027A
:1009700010D439F021D3009510959ADC202331232F
:1009800004C01AD395DC202B312B97DC20D3D2DB8B
:10099000BDD30081102F0AE108DCB8D311810BE12F
:1009A00004DC20C135D39A9937C0FDD2893200E0EA
:1009B0009007C8F3B1D3808191810A96EAE6F2E00C
:1009C00080839183ACD3ECE6F2E07CDCA5D303D347
:1009D000AAD3DCD3AAD474DC102F08E1E6DBAADBAF
:1009E00002DC40DC75D324E730E079D374D368DBD4
:1009F000ECE6F2E069D3EAE6F2E066D3E5E8F2E09D
:100A000063D326E830E06BD32FD8269600EC66D36C
:100A100057DB9A99F0C0FDCFD6D225E930E05FD3FD
:100A200023D85BD34DDB86DBF3D28F3000E0900719
:100A300008F0D8C0B8D2F9CF9B9969C0C4D276D398
:100A400061F4EDE8F2E0F5D20A3018F000E000932E
:100A50008D02102F02E1A9DBC4C079D359F47FD3F2
:100A600027D3F7DB223806E0300718F001E816E05C
:100A700029DC38D318DC59F4E4E8F2E0DED2093C92
:100A80001CF400E000938402102F07E18EDB00913C
:100A90009502023049F4EFE8F2E0CFD20F3F19F4AB
:100AA00000E000938F0226D300919502033049F4B1
:100AB000E0E9F2E0BED2023018F000E000939002CC
:100AC0001CD300919502043049F4E1E9F2E0B5D27B
:100AD0000F3F19F401E00093910212D300919502A7
:100AE000053049F4E4E9F2E0A4D2023018F000E065
:100AF0000093940208D32FD349F4EBE8F2E09DD29F
:100B00000F3F19F40FE000938B0261D26AC09C99E9
:100B100069C059D20BD359F4EEE8F2E08AD20A3018
:100B200018F000E000938E02102F03E194CF0FD352
:100B300061F4CBDB015010408CDB203403E0300744
:100B400018F400E413E0BEDBCDD2ADDB59F4E4E8E9
:100B5000F2E06FD208331CF000E000938402102F03
:100B600007E123DB00919502023049F4EFE8F2E05F
:100B700060D2033018F002E000938F02BBD20091E4
:100B80009502033049F4E0E9F2E053D2023018F064
:100B900000E000939002B1D200919502043049F434
:100BA000E1E9F2E046D2063018F005E00093910248
:100BB000A7D200919502053049F4E4E9F2E039D278
:100BC000023018F000E0009394029DD2C4D249F4A0
:100BD000EBE8F2E02ED2003118F000E000938B0237
:100BE000F6D1A8DA5BD237DB36952795A6D2020F6D
:100BF000131F19BD08BD9AD209F0A7C0369A05E0A7
:100C000007B904E610E0C5DADADA41DB40E050E08B
:100C100060E371E455D533D4E2E7F2E053DB00E062
:100C200007B995D211F404E407C0013011F403E4CC
:100C300003C0023019F407E40093970253DB38DB5A
:100C4000233600E0300759F4D2D140D20091970208
:100C50003FD228E731E043D207D726960DC0022FB6
:100C6000132F36D2C4D132D20091970231D22DE85F
:100C700031E035D2F9D6289630D222DA00919402AA
:100C8000002329F505D202D223D22CE431E027D269
:100C9000EBD62496B8D103C00FEF0EDA01968C0183
:100CA00020E030E0EAD328013901E6DAA801B901F1
:100CB0008201930173D508F032C1082F0154D9D9AC
:100CC000F6DA283C00E030073CF703E2E6CFE0D15B
:100CD000DDD1FED120E731E002D2C6D624960BE862
:100CE000FDD1EED92FE531E0FAD1BED600ECF6D138
:100CF000E7D9C2DAC4D3C801883000E0900708F011
:100D00008FEFB0DA0A5B1F4FE6E7F2E0DBDA312F54
:100D1000332332F04AE0C3DA0054ABD9082FCCD9E0
:100D2000C6DA293C00E030070CF4F9C0E6E7F2E04F
:100D3000B1D10F539ED905E0BFD9E6E7F2E0AAD1C1
:100D4000015497D905E0B8D9EAC0A0E000D209F073
:100D50004FC0ECE4F2E096D12BED31E0C0D1BBD135
:100D6000AFD95ED14F5F5F4FEED13A932A93B0D1A6
:100D700025ED31E0B4D178D6249609E8AFD1A0D9D9
:100D8000E8E5F2E07FD12BEC31E0A9D16DD62296D7
:100D900000ECA4D195D900919302005039F00A9546
:100DA00061F00A9589F00A95B1F01EC007EE21D1D5
:100DB0000AEA8ED121EC31E014C007EE1AD10AEA1A
:100DC00087D127EB31E00DC007EE13D10AEA80D1BD
:100DD0002DEA31E006C007EE0CD10AEA79D122EA09
:100DE00031E07DD141D6249609EC78D169D997C0FC
:100DF000013029F5F8D94FDA67D127E032E06FD119
:100E00006AD15ED92FDA64D12DEF31E068D12CD6CA
:100E1000229609E863D154D92CDA56D12DEE31E06F
:100E20005ED122D6229600EC59D14AD986D150D132
:100E300025EE31E054D118D622960BECD6CF0230F5
:100E400081F42BE331E04BD10FD647D139D9009152
:100E50008F02CFD021E132E042D106D6229600ECBB
:100E6000C4CF033091F42BE131E039D1FDD535D138
:100E700027D900919002002319F424E331E002C045
:100E80002CE231E02CD1F0D5EACF043061F429EF27
:100E900030E025D1E9D521D113D900919102A9D013
:100EA0002AE031E0D9CF053081F428EC30E017D1C9
:100EB000DBD513D105D900919402013019F42AEE43
:100EC00030E0E0CF29ED30E0DDCF063041F5009194
:100ED0008A02002321F126EA30E001D1C5D5FDD0F8
:100EE000EFD827EB30E08CD003C000E2E5D80196C4
:100EF000803100E0900750F4082F0054BAD806D192
:100F0000E6D9482F46D189F30FEFF0CF00918B023D
:100F10000058AFD80EE0ADD800E000938A020091EF
:100F20009002002319F0969A979A02C09698979883
:100F3000A395AD3108F4D2CA45D00093890203E6E7
:100F400010E093D9AED900918802002309F0C6CAF7
:100F50002FD0F0D801E000938802C0CA3CD90F53CB
:100F600011C039D90F53C4D902D10EC0FBD029D931
:100F700001D103D112D1F6D0089523D9F8D0C9C038
:100F80002AD90C53B5D9F6D001D162817381400FB3
:100F9000511F621F731FBEC01ED90C53E4CF1BD953
:100FA0000C53A6D9089508EE1DEFF3D801960895C5
:100FB000C1D808EE1DEFEDC801E010E040918B02B2
:100FC0008FD10895A0E001E000938702089501E029
:100FD00000938A020895208131810AE010E0129F77
:100FE000102D039F100D029F002D110D08950091EB
:100FF0008E0210E06DC0082F03BD08EB1BE00895C2
:1010000004E312E031D500EC34D804E312E058D800
:1010100080E090E008950DE605BD67D90081089550
:1010200000E816E928E930E09AD0B0D00895E5E963
:10103000F2E0008103950083089500810A95008302
:10104000089500831183EAE5F2E041D9EEE5F2E08C
:1010500041D9409191024ED9EEE5F2E040D920838A
:1010600031830895EEE4F2E032D9E2E5F2E032D9DC
:101070004091910211C02BD9228133814CED50E077
:1010800062D0089524D942E035D922C05A934A93B8
:10109000E2E7F2E01CD94AE02DD9089516D91BBD2C
:1010A0000ABD0895E2E8F2E012D980179107089589
:1010B0000ED90F5F1F4F08950AD9E6E5F2E00895B3
:1010C00006D9E2E6F2E0089502D902C000918D024D
:1010D0001A930A930895C8D4229600E8CAD704E365
:1010E00012E0089500E161D83AD00081102F01E1AB
:1010F0005CD80895102F04E158C8102F05E155C899
:10110000102F06E152C8102F09E14FC8EEE7F2E0B8
:10111000089533D042D00895EEE4F2E00895EAE570
:10112000F2E0D5D80895EAE5F2E00895009196023C
:10113000002308958C012DD0089500918402102F72
:10114000110F110B089560E070E040D108950091F7
:101150009502002308950091950206300895E0E875
:10116000F2E0089504B1202F30E015B10895E8E4CD
:10117000F2E00895E4E4F2E0089540815181628153
:101180007381401B510B620B730B08954081518199
:101190000895ACD001700023089540835183628389
:1011A000738308951DD3C801D9012A013B014CD096
:1011B00071F482019301F2D251F401E2E8E9F2E024
:1011C000008341830FEF1FEF2FE73FE73BC08C0108
:1011D0009D01A201B301BAD1AC01BD01DFD28C01E6
:1011E0009D0149F431D00BED1FE029EC10F03FE3F5
:1011F00029C03FEB27C0A201B30162D20801190147
:101200008201930121D08C019D01A0F4C7D28001FD
:10121000910148F085D3A801B9010BED1FE029E445
:1012200030E4CED10FC07CD34BED5FE069E470ECCD
:101230008DD108C0B3D28001910110F071D302C0EA
:101240006FD33058E8E0DDC240E050E060E070E08D
:10125000A5C209ED0DBF02E00EBFCAEDD3E05ED31B
:10126000002309F0DAD348D888D487C4BDD2DA0184
:1012700040E050E060E070E091D239F400E010E02E
:101280004D934C9320E030E00CC0B901660F771FFE
:101290007E57572F550F550B7D935C932F773078E2
:1012A0003F63E4E0B2C20024E8E0EA9532F0001FB8
:1012B000001C0416D0F3041AF8CF001F402D00952F
:1012C0000895FF27442312F4F1604195002312F49E
:1012D000F0950195E8DFF0FD0195F1FD4195089548
:1012E0004A951AF0000F111FFBCF08954A951AF086
:1012F00016950795FBCF089500241124EFE0001FF9
:10130000111F001C111C0416150610F0041A150AF2
:10131000EA95AAF7001F111F402D512D0095109539
:1013200008955195419550400895FF27552312F493
:10133000F160F7DF112312F4F09506D0DDDFF0FD48
:1013400003D0F1FDEECF0895119501951040089559
:1013500030952095109501951F4F2F4F3F4F0895C1
:1013600070956095509541955F4F6F4F7F4F0895F1
:101370004A952AF03695279517950795F9CF089540
:101380000024112422243324E0E2EA9592F0001F85
:10139000111F221F331F001C111C221C331C04169A
:1013A00015062606370688F3041A150A260A370A90
:1013B000ECCF001F111F221F331F402D512D622D16
:1013C000732D00951095209530950895FF2777236C
:1013D00012F4F160C5DF332312F4F095B9DFD0DFEA
:1013E000F69508F4B5DFF69508F4BACF0895FF270F
:1013F0001124770F1794660F7F1F09F008946795E3
:10140000EE270024330F0794220F3E1F09F00894A3
:101410002795089527FD0EC0EE0F001F111F221FF4
:101420003A953230B8F7332319F427FD31E002C082
:1014300027FF30E0E03811F400FF08940F4F1F4FF2
:101440002F4F3F4F323038F4332319F427FD31E06A
:1014500002C027FF30E03F3F09F4BBC0220F000C61
:10146000379527950895032E00200AF471DFE02FA9
:10147000012F122F232F3EE9D4CF0024F8CFC0DF55
:10148000432F4F5760F0403260F000202AF00FEFFA
:101490001FEF2FEF3FE7089530E8222797C033274B
:1014A000FCCF322F212F102F0E2F4F51419560DF8F
:1014B00007FE08954DCFE22FEF77E0301E070E07AD
:1014C0000895E62FEF77E0305E074E070895E32F8B
:1014D000EE0F27FBE0F9EF3F61F0EE2311F4EBDFB5
:1014E00029F0332398948894B8940895332318945A
:1014F000FACFE1DF19F00894B89403C0332388943D
:10150000389498940895E72FEE0F67FBE0F9EF3FCA
:1015100041F0EE2311F4D5DF11F07723E3CF7723E9
:10152000E6CFCFDF41F77723EACFEDDF70F029F484
:101530003723262F152F042F0895372FFACFE3DFF7
:1015400020F00BF008957327EAF747C0C0DFE8F3F7
:10155000B3F359F3D8DFC8F383F3A1F348DF40179F
:1015600051076207730778F0332E372F732D322E11
:10157000262F632D312E152F532D302E042F432D62
:10158000302C012C132C371739F066955795479559
:10159000F795E7957395F7CFEE0FE0E010245AF03A
:1015A000EF0F041F151F261F50F427951795079559
:1015B000E795339536CFEF0B040B150B260B31CF88
:1015C000E0E87E27C3CF302D30782227112700276F
:1015D00008953FE7302920E8F9CF302D3F672FEFFE
:1015E000F5CF91DF20F019F0707837270895F5CF07
:1015F0008ADFE8F3E3F37078372708959ECF372723
:101600003078E3CF64DF98F363F391F37CDF78F312
:10161000ABF3A9F3ECDE012407FA332311F07723AF
:1016200009F4D1CF3F577F57370F13F492F2CBCF46
:1016300031583F3FB1F34A923A9333242224112484
:10164000002433274424772720301207010789F02C
:1016500026951795079530F4040E451E361F171E64
:101660002E1E3F1E440F551F661F771FEE1FFF1FC4
:10167000EBCF732F399133203AF0000C441C771FC5
:10168000111C221C331C03C0339509F4A2CF7038FF
:1016900019F4402809F073954990232D122D012D3E
:1016A000E72F002407F8BDCE2EDF10F00BF09CCF03
:1016B00094CF29DFE9F3E0F3A2CF032E072689CFE9
:1016C00006DFB0F38BF3A9F31EDF90F3ABF3A9F3BE
:1016D0008EDE012407FA3F577F57371B3BF40AF091
:1016E00072CF303809F075CF315804C031583F3FC0
:1016F00009F469CF1124139440175107620728F0A9
:101700003A95000F111F221FEE1F3F3F21F4772350
:101710000AF45FCF58CF041B150B260BEF0B000FFD
:10172000111F221FEE1F77E17A95A2F0041715070B
:101730002607EF0730F0041B150B260BEF0B089460
:1017400001C08894111C221C331C000F111F221F82
:10175000EE1FEACF401751076207FE0718F021F489
:10176000E0E803C0EFEF01C0EE27012D122D232D7D
:1017700061CEC9DE80F013F473170895E32FEE0FE6
:1017800098940895731718940895BDDE20F0D1F34E
:10179000E0E8E727F4CF98948894089598DED8F38A
:1017A00043F399F3B0DEB8F39BF341F3E32FE7275C
:1017B0001AF4731798940895041715072607370726
:1017C000D1F33323BAF710F4889408950894089558
:1017D000FA92EA92DA92CA92BA92AA929A928A9269
:1017E0007A926A925A924A92BA93AA939A938A9355
:1017F0000895FF84EE84DD84CC84BB84AA8499841C
:1018000088847F806E805D804C80BB81AA819981B5
:101810008881F0E00FB6F894CE0FDF1F0FBE089559
:10182000DBDF229741E050E060E070E0B7DFC0F41A
:1018300040E0B4DF51F402E2E8E9F2E000835183D2
:101840000FEF1FEF2FE73FEF60C001E210E0E8E984
:10185000F2E0008311830FEF1FEF2FE73FE755C042
:10186000AE0104DDC801D90143EF54E065E37FE335
:1018700095DF68F4B7FBAA0FBB1FB395B695A79584
:10188000B7F908811981015010400883198340D0AD
:101890007FEB5CDE280139013BD07FE357DEA801F6
:1018A000B901820193010CDFC801D901A801B90176
:1018B000A9DE280139010881102F110F110B212FEA
:1018C000312FD1DD48E152E761E37FE39BDE480140
:1018D00059018201930142E252E964ED7EE392DE16
:1018E0004DED5BE96AE27FE331DEA201B3018ADEFE
:1018F00044E050E060E070E429DEAC01BD0182DE2E
:10190000A801B9018401950121DE2296ECE075CF92
:101910008C019D0140E050E060E8089501E00895E9
:1019200057DFC801D901BF773B2F41E050E060E8A5
:101930007FE334DF68F440E031DF29F40BED1FE092
:1019400029E43FE351C088249924AA24BB241CC065
:101950000BED802E0FE0902E09E4A02E0FE3B02EA9
:10196000082F40E07FEBF2DD280139018C019D0159
:1019700040E050E060E87FE3E9DDA801B9018201C1
:1019800093019EDEC801D9018C019D01AC01BD010E
:1019900039DE28013901640175014C015D0144E221
:1019A0005FEF6BE27CEB2EDE48E854E466EA7EE310
:1019B0001ED048E150EC6FE319D045EB1CD0C801B4
:1019C000D901820193014AEE54EB66E80FD046EB51
:1019D00012D0A801B9018C019D0172DEA401B501EC
:1019E00011DEA601B701B2DDE0E103CF70E4AEDDA8
:1019F000A201B30107CE5DEF68E670E4A7CD20E059
:101A000002D0E9F708952D9301501040202F212B8B
:101A100008952591F8DFE9F7089586E290E0FC014A
:101A200005911491FC013296A591B491FC01349674
:101A300025913491422F432B19F0F901EADF01C0BF
:101A4000DEDF069610E08233910748F30895CCDE7E
:101A5000F901A081B1810C93008111810F5F1F4FAB
:101A600000831183E4E0D1CEBFDE2497088319837D
:101A700089019E01285F3F4F2A833B83BE016E5F31
:101A80007F4FAE0127E23DE07BD020E0A881B98105
:101A90002C932496E4E0B9CE9FDE229748015901A9
:101AA00041E050E060E070E079DE98F440E076DEFE
:101AB00029F400E010E020E030E05CC001E210E03A
:101AC000E8E9F2E0008311830FEF1FEF2FE73FE714
:101AD00051C0AE01CBDBC801D90145EC53E062E453
:101AE0007FE334DD4AE151E562E17FE38BDD2801EC
:101AF0003901A801B9018C019D01E2DDA201B30108
:101B000025DD28013901088100FF15C008810A95EB
:101B100042E0D7DB802F042D43EF54E065EB7FE3F9
:101B200071DD37FB220F331F380F3695279537F9B4
:101B3000C801D9010CC0088142E0C3DBC201D30156
:101B4000B7FBAA0FBB1FB00FB695A795B7F98C01CD
:101B50009D0140E050E060E87EE354DD280139015A
:101B600084019501AC01BD01ABDDA801B901820181
:101B70009301ECDC2296ECE040CE00008895FECF8D
:101B800027DE2697088319832A833B834C835D8352
:101B90004B01CC24DD2401C0BDD0C0D005E2A0168D
:101BA00031F0AA20C9F786012696E0E122CE10E0A6
:101BB00000E02081285621F0245041F401E001C0CA
:101BC00011E09F012F5F3F4F28833983A7D02A2D33
:101BD000285509F46BC02B5059F02A9509F456C0CA
:101BE0002B50A9F0245049F0255009F45FC0D4CF00
:101BF000A5D0F801A0809CD0CFCFA0D0BAD098D0EB
:101C0000FC01A190CF01AA2041F284D0F9CF28E0B5
:101C100096D011F40023A1F5442420E8522E662426
:101C20007724112309F452C07FD009F04BC0A92FAB
:101C3000AA0FAA0BBA2F82D00E5F1F4F0083118309
:101C400004E6A01669F4BB235AF49095A095B095CC
:101C500081959F4FAF4FBF4F2C813D810DE273D0D7
:101C600002E0401600E050066006700608F448C026
:101C700084159505A605B70508F042C06CD0F0CFD5
:101C800044245524662400E4702E22C02AE057D054
:101C900011F4002321F420E1422E27E2BFCF442497
:101CA0000AEC502E0AE9602E0BE3EECF20E147D07C
:101CB00011F4002311F44424B1CF442455246624A4
:101CC00000E1E2CFA0E0B0E033D0CACF002339F08A
:101CD00035D04FD0A281B38131D00C5FAECF24D0AC
:101CE00089F7A5CF495F2C813D81042F2CD03CD0B2
:101CF000CA01DB0130D0012B022B032B09F44DCF9D
:101D000033D0402F405D4A3370F308E7A01651F7F7
:101D1000495DE9CF2C813D810A2D15C0E881F9810B
:101D2000A190E883F983089504E6A01626D021C087
:101D300024D00E5F1F4F0083118308951EC0E22E32
:101D4000FF2411230895EA81FB81099501E0C00E6B
:101D500000E0D01E089582019301A70160E070E0C9
:101D60000FDB2801390108958C019D01A201B30107
:101D700007CBF801808191810895F40100811181E0
:101D80000895257300726164696F646F6D2E7563C9
:101D90006F7A2E7275002A47726F756E642A20560C
:101DA00044493D2564202000256420583D256420B9
:101DB000593D256420200020202A2A2A2020302076
:101DC000202A2A2A20202000303132333435363779
:101DD00038392D3032343638002020202020202081
:101DE00020202020202020202000202020202D49DD
:101DF0006E642D20202020202020002D5644492BC9
:101E0000416D706C69747564652020002D4869739C
:101E1000746F6772616D2020202000202020202D0B
:101E200046696C7465722D20202020004B3D25648E
:101E300020202020202020202020202000202020C2
:101E400020202D4C65642D202020202020002D2DC9
:101E50002D4F464620002D2D2D4F4E200020202DA9
:101E6000566963652063686172742D20200020200C
:101E70002020202020202020202025642E256442A0
:101E80000020202020202049202020202020202049
:101E900020002025642E2564420025632D437525EE
:101EA000645F466525642020203C2D2D3E200025C2
:101EB000632D437525645F4665256420203C2564B9
:101EC0003E20200025633D31333525632020002549
:101ED000633D3930256320200025633D343525637B
:101EE00020200025633D30256320202000593D251A
:101EF00064202020202000663D25642000583D25D8
:101F0000642020202020002825642920202000642F
:101F1000593D25642020202020202020202000560C
:101F200044493D25642020200064583D256420203C
:101F30002020003D2564202020202020202020205B
:101F400020202020002A2A2A204B504F542D4D209B
:061F50002A2A2A202000CD
:00000001FF
